:1000000016C030C02FC02EC0A8C02CC02BC02AC024
:1000100029C028C027C026C025C024C023C000375F
:10002000003801010101010101020408102011241E
:100030001FBECFE5D2E0DEBFCDBF10E0A0E6B0E04E
:10004000EEE2F7E002C005900D92A436B107D9F7B1
:1000500020E0A4E6B0E001C01D92AF36B207E1F7A0
:10006000C3D063C3CDCF282F30E0F901E85DFF4F47
:100070009491F901EE5DFF4FE491EE23A1F081111F
:1000800013C08AB58F738ABDF0E0E05EFF4FA49184
:10009000B0E08FB7611113C0F8942C91E92FE0956F
:1000A000E223EC938FBF0895813019F48AB58F7CD9
:1000B000EACF843049F78CB58F7C8CBDE5CFF894BE
:1000C000EC91E92BEECF3FB7F89480916B009091C3
:1000D0006C00A0916D00B0916E002FB508B602FEC5
:1000E00005C02F3F19F00196A11DB11D3FBFBA2FCA
:1000F000A92F982F8827BC01CD01620F711D811D8A
:10010000911D42E0660F771F881F991F4A95D1F70E
:100110000895CF92DF92EF92FF92CF93DF936B011E
:100120007C01D1DFEB01C114D104E104F10439F405
:10013000DF91CF91FF90EF90DF90CF900895C3DFD4
:100140006C1B7D0B683E734070F381E0C81AD108C8
:10015000E108F108C851DC4FE6CF78941F920F9266
:100160000FB60F9211242F933F938F939F93AF93CA
:10017000BF938091670090916800A0916900B09151
:100180006A00309166002CE7230F2D3728F02FEFFF
:10019000230F0196A11DB11D209366008093670077
:1001A00090936800A0936900B0936A0080916B00FF
:1001B00090916C00A0916D00B0916E000196A11D10
:1001C000B11D80936B0090936C00A0936D00B09371
:1001D0006E00BF91AF919F918F913F912F910F90A2
:1001E0000FBE0F901F901895789480B7806880BFDD
:1001F00080B7806480BF8CB580648CBD8FEF8DBD6F
:1002000080B7807F876080BF89B7846089BF83B7EC
:10021000887F83BF8AB58C7F81608ABD83B7877FE3
:1002200083BF83B7887F836083BF86B1876086B9C9
:10023000379AE9E2F0E02491E3E2F0E0E491EE2382
:1002400089F08E2F90E0FC01E25EFF4FA491B0E0B8
:10025000805E9F4FFC0184918FB7F894EC91E22B64
:10026000EC938FBFEFE2F0E02491E9E2F0E0E4915B
:10027000EE23A1F08E2F90E0FC01E25EFF4FE491AF
:10028000AE2FB0E0805E9F4FFC0184918FB7F89451
:100290009C91E22FE095E923EC938FBF87B18F7299
:1002A00087B987B1807F816087B9369A3699FECF4A
:1002B00064B175B1809164009091650086179707CD
:1002C00024F47093650060936400809161009091C4
:1002D00062006817790724F47093620060936100EC
:1002E000C0916100D09162006C1B7D0B6F5F7F4FEE
:1002F000072E000C880B990BF9D06B017C016091E3
:100300006400709165006C1B7D0B6F5F7F4F072E43
:10031000000C880B990BEAD09B01AC01C701B60118
:100320004FD06B017C0180916000882309F441C0AB
:100330002FB7F8948091670090916800A0916900B0
:10034000B0916A002FBF80339547A105B10588F5AC
:1003500061E081E088DE20E030E048EC52E4C70153
:10036000B60154D195D0D5DE60E081E07CDE2DEC85
:100370003CEC4CEC5DE3C701B60144D11816E4F443
:1003800080916000811118C0CCE2D1E060E081E092
:100390006ADE61E081E067DE68EE73E080E090E0B5
:1003A000B8DE219799F762E370E080E090E0B1DE7B
:1003B00075CF10926000DBCF60E081E054DEF3CFB8
:1003C0000CD0E6C0DED040F0D5D030F021F45F3F55
:1003D00019F0C7C0511110C1CAC0EBD098F39923CE
:1003E000C9F35523B1F3951B550BBB27AA276217F9
:1003F0007307840738F09F5F5F4F220F331F441F3E
:10040000AA1FA9F333D00E2E3AF0E0E830D0915075
:100410005040E695001CCAF729D0FE2F27D0660F62
:10042000771F881FBB1F261737074807AB07B0E8A1
:1004300009F0BB0B802DBF01FF2793585F4F2AF0B7
:100440009E3F510568F08DC0D7C05F3FECF3983EEA
:10045000DCF3869577956795B795F7959F5FC9F714
:10046000880F911D9695879597F90895E1E0660F9D
:10047000771F881FBB1F621773078407BA0720F016
:10048000621B730B840BBA0BEE1F88F7E09508957F
:1004900098D088F09F5790F0B92F9927B751A0F0C6
:1004A000D1F0660F771F881F991F1AF0BA95C9F708
:1004B00012C0B13081F09FD0B1E008959CC0672F89
:1004C000782F8827B85F39F0B93FCCF386957795B8
:1004D0006795B395D9F73EF49095809570956195A1
:1004E0007F4F8F4F9F4F0895E89409C097FB3EF4CC
:1004F00090958095709561957F4F8F4F9F4F992371
:10050000A9F0F92F96E9BB279395F69587957795EE
:100510006795B795F111F8CFFAF4BB0F11F460FFAE
:100520001BC06F5F7F4F8F4F9F4F16C0882311F006
:1005300096E911C0772321F09EE8872F762F05C01A
:10054000662371F096E8862F70E060E02AF09A95B5
:10055000660F771F881FDAF7880F9695879597F9AA
:10056000089597F99F6780E870E060E008959FEF35
:1005700080EC089500240A9416161706180609063A
:10058000089500240A941216130614060506089509
:10059000092E0394000C11F4882352F0BB0F40F491
:1005A000BF2B11F460FF04C06F5F7F4F8F4F9F4FD1
:1005B000089557FD9058440F551F59F05F3F71F053
:1005C0004795880F97FB991F61F09F3F79F08795BA
:1005D0000895121613061406551FF2CF4695F1DF43
:1005E00008C0161617061806991FF1CF86957105D3
:1005F000610508940895E894BB2766277727CB0107
:1006000097F908956ED008F48FEF08950AD0C0CFFF
:10061000B1DF28F0B6DF18F0952309F0A2CFA7CFFD
:10062000EBCFC7DFA8F39923D9F35523C9F3950F6F
:1006300050E0551FAA27EE27FF27BB270024089468
:10064000679520F4E20FF31FB41F0A1E220F331F19
:10065000441FAA1F6695A9F7779530F4F30FB41FCE
:100660000A1E121E08F46395330F441FAA1F221F8F
:10067000769599F7879520F4B40F0A1E121E631F12
:10068000440FAA1F221F331F8695A9F7862F712DAD
:10069000602D11249F5750408AF0E1F088234AF0E2
:1006A000EE0FFF1FBB1F661F771F881F9150504022
:1006B000A9F79E3F510570F054CF9ECF5F3FECF3FA
:1006C000983EDCF3869577956795B795F795E7950E
:1006D0009F5FC1F7FE2B880F911D9695879597F91F
:1006E0000895990F0008550FAA0BE0E8FEEF1616C3
:1006F0001706E807F907C0F012161306E407F50716
:1007000098F0621B730B840B950B39F40A2661F089
:10071000232B242B252B21F408950A2609F4A1402C
:0E072000A6958FEF811D811D0895F894FFCFDF
:04072E0001FF7F0048
:00000001FF
